:020000040000FA
:06000000C0EF07F0120042
:0600080004EF10F01200ED
:060018000CEF10F01200D5
:02002A000000D4
:04002C00040110516A
:10003000600BE842E842E842E842E842000901E099
:1000400055D01151070A51E00B0A4FE0070A40E072
:10005000010A2CE00B0A28E0020A26E0030A22E04B
:10006000080A12E0010A0EE00F0A0AE0030A01E0A2
:100070003CD00001010EB06F0001040EB76F36D006
:1000800036D834D090D832D00001010EB06F0001C4
:10009000B90EB16F000EB26F0001B8930001010EEE
:1000A000B56F24D0A8D822D0F5D820D00001010EF9
:1000B000B06F040114510001B16FB26BBA0EB127D9
:1000C000000EB2230001B8930001010EB56F0ED0EF
:1000D0000001010EB06F04011451EA6ABA0FE96E13
:1000E000000EEA2212C4EFFF01D000D01200800EF1
:1000F0000401105D57E11351030A34E0010A10E0D6
:10010000030A01E04DD00001010EB06F0001700E36
:10011000B16F0C0EB26F120E0001B56FB66B40D00E
:100120000001010EB06F04011251F66EF76AD8900B
:10013000F636F736B00EF6260D0EF7220900F5CF8B
:10014000B1F00A00F5CFB2F0020E0001F76AB12556
:10015000F66EB251F7220900F5CFB5F00A00F5CFDF
:10016000B6F01ED00001010EB06F04011251F66E00
:10017000F76AD890F636F736B40EF6260D0EF7224B
:100180000900F5CFB1F00A00F5CFB2F0B1C0F6FF2B
:10019000B2C0F7FF0800F5500001B56FB66B00D094
:1001A0000001B88312000001010EB06F0F0EE66E61
:1001B000710EE66E0F0EE66E23EC06F0E552E55288
:1001C000E552010EE66EBA0EE66E000EE66E23EC08
:1001D00006F0E552E552E55212C4B9F0040112519D
:1001E00004E10001050EB76F05D00001060EB76FE0
:1001F000EFEC04F012000401186B196B04011051AC
:100200001F0B020A15E0030A0FE0010A01E034D0D7
:100210000001010EB06F02D0040118810001B8A1E5
:1002200002D00401188328D00001010EB06F24D041
:100230000001010EB06F040114510F0B080DF350B3
:10024000016A000F006E040E01221451800B01E0C0
:10025000010E040DF35000010024B36F000E0120C5
:10026000B46FB3C0E9FFB4C0EAFFEF50040B03E082
:100270000401010E186F00D00001B0050AE1000171
:10028000180EB16F040EB26F0001B8930001020E98
:10029000B56F12000401120510E110511F0B000987
:1002A0000CE10001010EB06F030E0401115D03E1CA
:1002B0000001B88102D00001B891040112513AE165
:1002C00010511F0B020836E114510F0B000932E0E8
:1002D0000001010EB06F040114510F0B080DF35013
:1002E000016A000F006E040E01221451800B01E020
:1002F000010E040DF35000010024B36F000E012025
:10030000B46F030E0401115D07E1840EB3C0E9FF71
:10031000B4C0EAFFEF6E0ED014AF06D0B3C0E9FF51
:10032000B4C0EAFFEF6A06D0880EB3C0E9FFB4C0DC
:06033000EAFFEF6E12006F
:0A0336006C500BE1040100513C0B78
:10034000E842E8420D0802E108D801D03CD804D0C8
:10035000040E6C5C01E147D81200D9CFE6FFE1CF73
:10036000D9FFE6520001AF6BB06BB56BB66B16EC04
:1003700000F0DF6ADF50006E016A010E005C000EC3
:1003800001581BE20001B05101E017D0F76ADF34D9
:10039000FE0BF736F66EBE0EF6260D0EF72209009E
:1003A000F5CF00F00800F5CF01F004D001C0FAFF4E
:1003B0000050F96EFBDFDF2ADDD7DDD8E552E552CC
:1003C000E7CFD9FF1200020E0001AF5D0AE196D817
:1003D000040100BD03D0C80E006F02D0880E006F6C
:1003E00001D00FD91200040E0001B75D0AE112C45A
:1003F0006EFF6E50000803E2050EB76F02D0030EC9
:10040000B76F0001AF050AE10BD8040104BD03D0AA
:10041000C80E046F02D0880E046F01D0F2D812000B
:10042000D9CFE6FFE1CFD9FF020EE1260001080E89
:10043000B55D000EB65905E2B5C0DEFFB6C0DDFF02
:1004400003D0080EDE6EDD6A040104930491010EF0
:10045000DB500413DFCF05F4000EDB500001B55F65
:10046000010EDB50B65B180EB36F040EB46F0001C3
:10047000B8A31ED0D9CFE9FFDACFEAFFEE50ED10D6
:1004800016E0B1C0F6FFB2C0F7FF0800F550B3C0E8
:10049000E9FFB4C0EAFFEF6E0001B32B000EB423F6
:1004A000B12BB223DF06010E01E2DB06E3D71CD03D
:1004B000D9CFE9FFDACFEAFFEE50ED1015E0B1C079
:1004C000E9FFB2C0EAFFEF50B3C0E9FFB4C0EAFFF2
:1004D000EF6E0001B32B000EB423B12BB223DF0665
:1004E000010E01E2DB06E4D7020EE15C02E2E16A02
:1004F000E552E16EE552E7CFD9FF1200D9CFE6FF12
:10050000E1CFD9FF020EE126030E04010015E76ECC
:10051000010EE7CFDBFF01C4DFFFDE500001B5278E
:10052000DD50B623180EB16F040EB26FD9CFE9FFBC
:10053000DACFEAFFEE50ED1014E0B1C0E9FFB2C02F
:10054000EAFFEF50B3C0E9FFB4C0EAFFEF6EB32B90
:10055000000EB423B12BB223DF06010E01E2DB064D
:10056000E5D7020EE15C02E2E16AE552E16EE55296
:10057000E7CFD9FF12006D980001B0510CE10401E2
:10058000080E016F100E026F040E036F840E006FD1
:100590000401046F35D0040110AF22D00001B55121
:1005A0000401165D0001B6510401175904E216C496
:1005B000B5F017C4B6F034DF0001010EAF6F0401CF
:1005C000080E016F100E026F040E036F800E006F95
:1005D0000401180E066F040E076FC80E046F10D0CA
:1005E0000001020EAF6F0401056BC80E046F040119
:1005F000080E016F180E026F040E036FC80E006F15
:1006000012000001AF6B0401080E016F100E026FA3
:0E061000040E036F880E006F0401046B1200CD
:02061E00550E77
:10062000A76EAA0EA76EA68212000001420E6A6F84
:10063000020E6B6F010E6C6F12000001606B665151
:10064000605D1EE260C000F0016A026A675100242A
:10065000F36E68510120F46E69510220F86EF4CFF8
:10066000F7FFF3CFF6FF0800F5CF61F06051EA6ABB
:100670006A0FE96E000EEA2261C0EFFF602BDFD740
:10068000F86A1200840EA66E0001606B6651605D10
:1006900027E26051EA6A6A0FE96E000EEA22EFCFA4
:1006A00003F060C000F0016A026A67510024F36E33
:1006B00068510120F46E69510220F86EF4CFF7FF03
:1006C000F3CFF6FF03C0F5FF0C001F0E60151F08E7
:1006D00003E06605605D01E1A2DF0001602BD6D773
:1006E00012000001606B6651605D20E2940EA66E00
:1006F0006051006E016A060ED89000360136E8049B
:10070000FBE1026A01BE0268000167510024F36E3A
:1007100068510120F46E69510220F86EF4CFF7FFA2
:10072000F3CFF6FF7CDF0001602BDDD7F86A120003
:10073000A66A0001606B6651605D0EE2675160253C
:10074000A96EA6806051EA6A6A0FE96E000EEA227D
:10075000A8CFEFFF602BEFD712000001606B66514E
:10076000605D13E267516025A96E6051EA6A6A0F05
:10077000E96E000EEA22EF50A86E040EA66E4FDF5F
:10078000A6B2FED70001602BEAD71200C40EA66EF7
:100790000001606B6651605D20E26051EA6A6A0F99
:1007A000E96E000EEA22EFCF03F060C000F0016AAC
:1007B000026A67510024F36E68510120F46E69519A
:1007C0000220F86EF4CFF7FFF3CFF6FF03C0F5FF7A
:1007D0000C0025DF0001602BDDD7F86A1200400E07
:1007E000E66E650EE66E000EE66E3EEC05F0E55236
:1007F000E552E552000870E20001606B00016551AE
:10080000FF0A57E0FA0A50E0010A3BE0070A34E029
:10081000010A2DE0030A18E0070A16E0700A01E059
:100820005AD003DF0001040E606F04010CBFFDD736
:10083000400EE66E650EE66E000EE66E04EC05F008
:10084000E552E552E55248D0F8DE050E000160277A
:1008500004010CBFFDD7400EE66E650EE66E000E7D
:10086000E66E04EC05F0E552E552E55235D00ADFBC
:100870000001010E606F30D034DF0001010E606FA7
:100880002BD056DF050E0001602704010CBFFDD7F9
:10089000400EE66E650EE66E000EE66E04EC05F0A8
:1008A000E552E552E55218D058DF0001010E606FA5
:1008B00013D09BEC05F00001636B646B00016307D0
:1008C000000E645B00016351641103E0000000004E
:0A08D000F5D7FF0001D000D01200A0
:0608DA00040110511F0B88
:1008E000010801E079D0145101E076D0060E115DC7
:1008F0002EE11351230A28E0010A13E0030A01E064
:1009000024D00001020EB06F0001B90505E100011D
:10091000940EB16F0C0EB26F090E0001B56FB66B7D
:1009200014D00001020EB06F0001B90505E100010D
:10093000930EB16F0D0EB26F0001B90504E11D0EEB
:100940000001B56FB66B01D000D00001B88304017F
:100950001051600BE842E842E842E842E8420108F0
:1009600001E03AD011510B0A31E0080A21E0090AEE
:1009700019E0080A09E00B0A05E0080A01E02CD09A
:100980002CD82AD02BD828D00001020EB06F00013D
:10099000BB0EB16F000EB26F0001B8930001010EE3
:1009A000B56F1AD00001020EB06F13C4BBF014D0A3
:1009B0000001020EB06F0001BC0EB16F000EB26FED
:1009C0000001B8930001010EB56F06D00001020EC0
:1009D000B06F12C4BCF000D012001200120000016F
:1009E000BD6B1E0E716E0401400E096F200E0A6F62
:1009F000040E0B6F880E086F0401600E0E6F040E5C
:100A00000F6F400E0C6F1200D9CFE6FFE1CFD9FF78
:100A1000E652FC0EDB50400805E2400EF36EFC0E81
:100A2000F3CFDBFFDF6AFC0EDB50DF5C19E2DF5047
:100A3000E76EFD0EDBCFE9FFFE0EDBCFEAFFE750EE
:100A4000E926000EEA22EF50E66EDF50EA6A600FF8
:100A5000E96E040EEA22E552E750EF6EDF2AE3D793
:100A6000FC0EDBCF0DF4400E04010C170C7D880E3C
:100A70000C13E552E552E7CFD9FF1200D9CFE6FFBC
:100A8000E1CFD9FF0001BD6B040108BF30D0FC0EDF
:100A9000DBCF00F00951D880005403E2FC0E09C4FA
:100AA000DBFF0001BD6BFC0EDB50BD5D19E2BD51EB
:100AB000EA6A200FE96E040EEA22EF50E66EBD519D
:100AC000E76EFD0EDBCFE9FFFE0EDBCFEAFFE7505E
:100AD000E926000EEA22E552E750EF6EBD2BE3D780
:100AE0000401400E096F0817087D880E08130001E5
:0C0AF000BD5100D0E552E7CFD9FF120045
:040AFC006DA60FD8FC
:100B000002D06DB613D80001B70508E16DBA06D062
:100B1000686A696A69806988020EB76F12006D6A37
:100B2000696A6D860001010EB76F12006D6A696A0D
:100B30000001B76B120096EF05F00001B75101E11B
:100B40003AD06850040B04E06950040B01E038D837
:100B50006DB231D06850010B04E06950010B01E027
:100B600050D86850100B04E06950100B01E024D8F5
:100B70006850400B04E06950400B01E037D86850E2
:100B8000200B04E06950200B01E032D86850020BC2
:100B900004E06950020B01E032D8030E0001B75D9A
:100BA00001E209D06850080B06E06950080B03E029
:100BB0009BEC01F068961200698468986D821200BF
:100BC0006D926994689412000001B8A10ED0F8DF0C
:100BD0006D840001080EBE6F070EBF6FBE07000ECA
:100BE000BF5BBE51BF11FAE16D941200689C120008
:100BF00070A003D001EC03F07090689A1200689224
:100C000012006A6A686A9F0E6B6E7B0E696E6E6A6E
:100C10000F0EE66E710EE66E0F0EE66E14D8E552FC
:100C2000E552E552160E706E68A602D06896FCD7A3
:100C30006D9801EC03F00001B8910001B96B00015F
:100C4000030EB76F1200D9CFE6FFE1CFD9FFFD0E3B
:100C5000DBCFE9FFFE0EDBCFEAFFFC0EDB5004E04A
:100C6000EE6AFC0EDB06F9D7E552E7CFD9FF12009A
:100C70001201000200000008D80433000100010244
:100C80000302090229000101028032090400000266
:100C900003000000092101000001221D0007058159
:100CA0000340000107050103400001090220000183
:100CB000020480320904000002FF000000070581E1
:100CC0000340000107050103400001040309043447
:100CD000034D006900630072006F006300680069E3
:100CE000007000200054006500630068006E006F13
:100CF000006C006F0067007900200049006E0063FF
:100D0000002E0048035000490043006B0069007446
:100D1000002000320020004D006900630072006F67
:100D20000063006F006E00740072006F006C006C56
:100D300000650072002000500072006F00670072B2
:100D40000061006D006D00650072001603500049DF
:100D500000430031003800460032003500350030D5
:100D60000032035000490043006B0069007400200A
:100D7000003200200043006F006E006600690067CB
:100D800000750072006100740069006F006E002041
:100D90000032000600FF0901A101190129401500D8
:100DA00026FF00750895408102190129409102C073
:100DB000820CAB0CCB0CCF0C030D4B0D610DDA0884
:100DC000D9CFE6FFE1CFD9FF040EE126938A818ACD
:100DD000F19E580EE66EA9EC07F0E55281AA3BD0D1
:100DE000FE0EF66E7F0EF76EF86A0800F550DF6EA5
:100DF000550EDF5C30E14CD8030EDB6A54D8D95075
:100E0000010FE96EDACFEAFFEE50ED101EE18B70B4
:100E1000030EDB2A030EDB50020817E19BEC05F002
:100E2000010EDB6A020EDB6A010EDB06DBCF00F08F
:100E3000020E01E2DB06DBCF01F00050011003E0FF
:100E400000000000F1D700EF10F0010EDB06020EEB
:100E500001E2DB06D3D71CD826D8EFEC03F0D9503B
:100E6000010FE96EDACFEAFFEE50ED1001E18B7071
:100E7000010EDB06020E01E2DB06EED7040EE15C9A
:100E800002E2E16AE552E16EE552E7CFD9FF1200D6
:100E9000140E6F6E0001B76B0001B86B0001B96BE7
:100EA0008B90949012007EEC05F06FBE02D09DEC0A
:040EB00005F0120037
:0C0EB4002A0EF66E000EF76E000EF86EAF
:100EC00000010900F550AA6F0900F550AB6F03E16E
:100ED000AA6701D03DD00900F550A56F0900F55073
:100EE000A66F0900F550A76F09000900F550E96EDB
:100EF0000900F550EA6E090009000900F550A86FD5
:100F00000900F550A96F09000900F6CFACF0F7CF42
:100F1000ADF0F8CFAEF0A5C0F6FFA6C0F7FFA7C0B2
:100F2000F8FF0001A85302E1A95307E00900F550BA
:100F3000EE6EA807F8E2A907F9D7ACC0F6FFADC07E
:100F4000F7FFAEC0F8FF0001AA07000EAB5BBFD7EA
:020F500012008D
:0E0F5200FF0EE350076EEF0E01D0F30EE76EB8
:100F6000E72EB0EF07F00C0E066EE76AE72EB6EF3D
:100F700007F0062EB5EF07F0072EAEEF07F01200D0
:100F800013EE00F023EE00F0F86A059C5AEC07F02F
:080F9000E0EC06F0FDD71200B1
:020000040030CA
:0100000024DB
:010001000EF0
:0100020038C5
:010003001EDE
:0100050001F9
:010006008178
:010008000FE8
:01000900C036
:01000A000EE7
:01000B00A054
:01000C000FE4
:01000D0040B2
:00000001FF
